:06000000020FD602006BA6
:03000B0002006B85
:0300130002006B7D
:03001B0002006B75
:0300230002006B6D
:03002B0002006B65
:0300330002006B5D
:03003B0002006B55
:0300430002006B4D
:03004B0002006B45
:0300530002006B3D
:03005B0002006B35
:0300630002006B2D
:01006B003262
:1000800002006B0002006B0002006B0002006B00BC
:1000900002006B0002006B0002006B0002006B00AC
:1000A00002006B0002006B0002006B0002006B009C
:0800B00002006B0002006B006E
:1001000002006B0002006B0002006B0002006B003B
:1001100002006B0002006B0002006B0002006B002B
:1001200002006B0002006B0002006B0002006B001B
:1001300002006B0002006B0002006B0002006B000B
:1001400002006B0002006B0002006B0002006B00FB
:1001500002006B0002006B0002006B0002006B00EB
:1001600002006B0002006B0002006B0002006B00DB
:1001700002006B0002006B0002006B0002006B00CB
:10018000438080C28122C01A85811AAA8253807F4F
:10019000E51A24FBF88682C002120277D002E51A23
:1001A00024FCF8746056FB602CBB20028005BB4029
:1001B0001F800CA81A181818868212027780168AD7
:1001C00082120277A81A1818188682120277800500
:1001D0007582018025E51A24F8F8E66017E51A24EF
:1001E000F8F8E6C0E0E51A24F9F88682088683125A
:1001F000033B1581438080758200D01A22C01A8586
:10020000811AAA8253807FE51A24FBF88682C002F5
:10021000120277D002E51A24FCF8746056FB602FB6
:10022000BB20028005BB401F800CA81A1818188636
:100230008212027780198A82120277A81A18181877
:10024000868212027780084380807582018025E5CE
:100250001A24F8F8E66017E51A24F8F8E6C0E0E595
:100260001A24F9F886820886831202C81581438011
:1002700080758200D01A22E58223FA139281D280FF
:10028000C280EA23FA139281D280C280EA23FA1351
:100290009281D280C280EA23FA139281D280C280F6
:1002A000EA23FA139281D280C280EA23FA13928160
:1002B000D280C280EA23FA139281D280C280EA23DC
:1002C000139281D280C28022C01A85811AAA82AB81
:1002D00083A81A18181886048C051CED601E8A82E3
:1002E0008B83E0FDA3AA82AB838D82C002C003C0D2
:1002F00004120277D004D003D00280DCD01A22E4AA
:10030000D280A28333C280D280A28333C280D280C3
:10031000A28333C280D280A28333C280D280A283E0
:1003200033C280D280A28333C280D280A28333C200
:1003300080D280A28333C280F58222C01A85811ABE
:10034000AA82AB83A81A18181886048C051CED60C5
:10035000121202FFAD828A828B83EDF0A3AA82ABD8
:060360008380E8D01A22A0
:030FDC00020FE41D
:030FF700020FDF07
:050FDF001206A080FED7
:10036600C200E4F508F509F50AD201750B00750C13
:100376000012088512088275CB6375CAC0758E0097
:1003860075C804D2AFD2B0D2B190E60B7403F000B8
:1003960090E61074A0F00090E61174A0F00090E6CC
:1003A6001274A2F00090E61474E3F00090E615745F
:1003B600A0F00090E6137420F00090E6047480F03C
:1003C6000090E6047482F00090E6047484F00090D5
:1003D600E6047486F00090E6047488F00090E60463
:1003E600E4F00090E6497482F00090E6497482F0E9
:1003F6000090E6497488F00090E6497488F0009011
:10040600E60BE4F00090E618E4F00090E619E4F05C
:100416000090E61A7408F00090E61B7410F0009045
:10042600E6267402F00090E627E4F00090E60274F7
:10043600EBF00043B0100022AA82850C827583E09F
:10044600EAF0050C0509E4B50902050A22C01AE519
:1004560081F51A2404F58120000302061B12088187
:1004660090E6A2E0FA30E1030204F7E509450A60E6
:10047600687AC07BE78B9D7AC07BE77B008A9E907B
:10048600E67C7431F07460F0C3743E9509E4950A15
:1004960050107A3EE50924C2F509E50A34FFF50A4B
:1004A6008007AA09E4F509F50A8A037C007DE08D38
:1004B6009A850B9B8A041AEC601090E67BE090E626
:1004C6007CF07C007DE08D9A80EA859B0B0090E6AF
:1004D6008F74022BF0D2CF801830CF1590E7C074FE
:1004E60031F090E7C17460F00090E68F7402F0C2BC
:1004F600CFE5AA30E00302061BC3E50994C1E50A6D
:100506009400400302061B90E690E0FB7A0090E61A
:1005160091E07D004202ED4203A81A080808A602EF
:1005260008A6037C007DF08D9A7C007DF07D008C12
:100536009BA81A08E4F608F6A81A08A91A090909D0
:10054600C3E69708E609974003020614E508700318
:100556000205DCA81A080808A91A09E6C397FE08C6
:10056600E60997FFAA087B00C3EA9EEB9F50048A20
:10057600068B078E02E508C39AF508A81A08EE2628
:10058600F6EF0836F63001248E028F038A048B05B7
:100596001ABAFF011BEC4D609F90E67BE0F582C026
:1005A60002C0031208C9D003D00280E08E028F0376
:1005B6008A048B051ABAFF011BEC4D700302053E37
:1005C60090E67BE0F582C002C00312090612043EE3
:1005D600D003D00280DA90E67BE0FA23235401FBB5
:1005E600B401009201EA30E707743F5AF508801219
:1005F6003001078A8212089F80088A821208BB127D
:10060600043EA81A0806B60002080602053E009037
:10061600E6917480F0851A81D01A2290E6B8E0FA45
:1006260020E70C90E6B9E07002D2007582012290B4
:10063600E6B9E0FABA902B90E6BCE025E0547FFAE2
:100646002400F582E43418F583E0FB90E740F0EAF5
:10065600042400F582E43418F583E0FA90E741F0CB
:10066600800C90E7407436F090E7417483F090E692
:100676008AE4F090E6BEE0FABA0200500790E6BEC1
:10068600E0FA80027A0290E68BEAF0758201223067
:100696000203120B3912045380F5C2AF120366121D
:1006A60006FC120F09120AA3D2AF12099802069588
:10E100001201100100000040FB090160000401023F
:10E1100003010A061001FFFFFF400100090237005A
:10E12000020100804B0904000002FFFFFF02070507
:10E1300081024000000705020240000009040100BE
:10E1400002FFFFFF02070586020002000705080222
:03E15000000200CA
:10E154001201100100000040FB09016000040102EB
:10E1640003010A061001FFFFFF4001000902370006
:10E17400020100804B0904000002FFFFFF020705B3
:10E18400810240000007050202400000090401006A
:10E1940002FFFFFF02070586024000000705080290
:10E1A40040000004B0E1B6E1C4E1DCE10603000094
:10E1B40009040E0341006C007400650072006100E4
:10E1C40018035500530042002D0042006C0061000A
:10E1D40073007400650072001203300030003000D8
:0AE1E4003000300030003000300041
:1006B600AA82E50D54FEFBB50D0280298A048C053D
:1006C600E4620EED620FEB2400F582E43418F58344
:1006D600E0FB7C00620EEC620FE50E33C50F33C5FE
:1006E6000F92E0F50EAB0D050DEB2400F582E43418
:1006F60018F583EAF022750D00750EAA750FAA7516
:1007060082001206B67582001206B67A00C3EA6443
:100716008094865017EA2408F582E434E1F583E0F4
:10072600F582C0021206B6D0020A80E17A00C3EA58
:10073600648094825017EA2423F582E434E1F58339
:10074600E0F582C0021206B6D0020A80E175821C6C
:100756001206B67582001206B67A00C3EA64809461
:10076600825017EA2402F582E434E1F583E0F5824B
:10077600C0021206B6D0020A80E17486250DFAF58B
:1007860082C0021206B690E1B6E0F5821206B6D035
:100796000290E1B6E02AFAF582C0021206B690E1AE
:1007A600C4E0F5821206B6D00290E1C4E02AF582D2
:1007B6001206B690E1DCE0F5821206B67A0090E108
:1007C600B6E0FBC3EA64808BF063F08095F05017C7
:1007D600EA24B6F582E434E1F583E0F582C002123C
:1007E60006B6D0020A80D77A0090E1C4E0FBC3EADD
:1007F60064808BF063F08095F05017EA24C4F5828C
:10080600E434E1F583E0F582C0021206B6D0020AAE
:1008160080D77A0090E1DCE0FBC3EA64808BF0636A
:10082600F08095F05017EA24DCF582E434E1F58394
:10083600E0F582C0021206B6D0020A80D77A00C35B
:10084600EA648094845017EA240EF582E434E1F5D4
:1008560083E0F582C0021206B6D0020A80E17482F5
:10086600250D40087582001206B680F2AA0E901871
:100876007EEAF0AA0F90187FEAF022222222229026
:10088600E6007412F090E60174E3F0AAB574FE5A1D
:10089600F5F0741E45F0F5B522E582FA1392B2EA38
:1008A600A2E192B1EAA2E492B3EAA2E5E433FAB491
:1008B600010092B42212089FA2B0E433FA74024AED
:1008C600F58222E5821392B3D2B213C2B292B3D2A8
:1008D600B213C2B292B3D2B213C2B292B3D2B213AD
:1008E600C2B292B3D2B213C2B292B3D2B213C2B2EE
:1008F60092B3D2B213C2B292B3D2B200C2B2222221
:10090600E582A2B01392B3D2B2C2B2A2B01392B32E
:10091600D2B2C2B2A2B01392B3D2B2C2B2A2B013D2
:1009260092B3D2B2C2B2A2B01392B3D2B2C2B2A240
:10093600B01392B3D2B2C2B2A2B01392B3D2B2C2C1
:10094600B2A2B01392B3D2B2C2B2F582222278809A
:10095600E84400600C7901901800E4F0A3D8FCD9B3
:10096600FAD083D082F6D8FDC082C0837582002279
:1009760090E6A0E04401F022AA8274805AC423546F
:100986001FFB740F5A90E6834BF090E683E04420F9
:10099600F02290E680E0440AF09000FA120FC5902B
:1009A600E65D74FFF090E65F74FFF05391EF90E61A
:0609B60080E054F7F0227E
:060FF100E478FFF6D8FDD4
:060FD6007510007511000A
:1009BC0090E680E0FA30E7267512007513E17514A5
:1009CC00127515E175161C7517E17518707519E11E
:1009DC0090E6267402F00090E627E4F000227512EF
:1009EC00547513E17514667515E17516707517E17C
:1009FC0075181C7519E190E626E4F00090E6277452
:100A0C0040F000225391EF75A100D20232C021C0F8
:100A1C00E0C0F0C082C083C002C003C004C005C0E7
:100A2C0006C007C000C001C0D075D0005391EF754F
:100A3C00A1001209BCD0D0D001D000D007D006D074
:100A4C0005D004D003D002D083D082D0F0D0E0D037
:100A5C002132C021C0E0C0F0C082C083C002C003FC
:100A6C00C004C005C006C007C000C001C0D075D00E
:100A7C00005391EF75A1001209BCD0D0D001D00069
:100A8C00D007D006D005D004D003D002D083D082BA
:100A9C00D0F0D0E0D021321209BC751B10751C0AA5
:100AAC00758200120E62751B19751C0A7582101264
:100ABC000E62751B5E751C0A758214120E6290E62E
:100ACC005C7431F022E582547FFA24F7500475826D
:100ADC000022BA010475820122530201E4BA00011A
:100AEC0004F58222AA82BA010C90E6A1E0FB7C00FC
:100AFC008B828C8322BA810C90E6A2E0FB7C008B6B
:100B0C00828C832253027FEA700C90E6A0E0FB7C7F
:100B1C00008B828C832290E6A3E0FB7C00EAC3135B
:100B2C00FA7D00EA2BFBED3C8B82F58322C202900E
:100B3C00E6B8E0FA530260BA00028028BA200280BC
:100B4C000DBA4002800EBA60028003020DF7120942
:100B5C0076020DF7120621E5826003020DF71209E9
:100B6C0076020DF790E6B8E0FA530280BA80028064
:100B7C0003020CF890E6B9E0FABA0003020C71BA61
:100B8C0006028035BA08028008BA0A028017020CE5
:100B9C00F290E740E510F090E68AE4F090E68B7472
:100BAC0001F0020DF790E740E511F090E68AE4F0D1
:100BBC0090E68B7401F0020DF790E6BBE0FABA01F7
:100BCC00028017BA02028038BA03028059BA0602B0
:100BDC00801BBA0702803C020C6BAA12AB1390E686
:100BEC00B3EBF07B0090E6B4EAF0020DF7AA14AB7D
:100BFC001590E6B3EBF07B0090E6B4EAF0020DF74B
:100C0C00AA16AB1790E6B3EBF07B0090E6B4EAF0D3
:100C1C00020DF7AA18AB1990E6B3EBF07B0090E647
:100C2C00B4EAF0020DF790E6BAE0FA90E1A7E0FB27
:100C3C00C3EA9B4006120976020DF790E6BAE075FE
:100C4C00F002A424A8F58274E135F0F583E0FAA350
:100C5C00E090E6B3F07B0090E6B4EAF0020DF712F8
:100C6C000976020DF790E6B8E0FA53021FBA0002BB
:100C7C00800ABA0102801BBA0266802C90E740E41D
:100C8C00F090E741F090E68AF090E68B7402F00267
:100C9C000DF790E740E4F090E741F090E68AF09091
:100CAC00E68B7402F0020DF790E6BCE0F582120AB6
:100CBC00D1E582602590E6BCE0F582120AF0E0FAFC
:100CCC0053020190E740EAF090E741E4F090E68AA5
:100CDC00F090E68B7402F0020DF7120976020DF714
:100CEC00120976020DF7120976020DF790E6B9E0BB
:100CFC00FA24F45003020DF4EA2A2A900D0B730225
:100D0C000DF4020D41020DBC020D9D020DF4020DFD
:100D1C00F4020DF4020DF4020DF4020D2F020DF489
:100D2C00020D3890E6BAE0F510020DF790E6BAE045
:100D3C00F511020DF790E6B8E0FA53021FBA000263
:100D4C008005BA0247800A90E6BAE0120976020DD5
:100D5C00F790E6BAE0703090E6BCE0F582120AD16A
:100D6C00E582602390E6BCE0F582120AF0AA82AB21
:100D7C0083E0FC5304FE8A828B83ECF090E6BCE0AB
:100D8C00F58212097E8064120976805F12097680E2
:100D9C005A90E6B8E0FA53021FBA004F90E6BAE058
:100DAC00FABA01028005BA02028040120976803B31
:100DBC0090E6BAE0FA702C90E6BCE0F582120AD10B
:100DCC00E582601A90E6BCE0F582120AF0AA82ABCA
:100DDC0083E0FC4304018A828B83ECF0800D1209C2
:100DEC00768008120976800312097690E6A0E0441A
:100DFC0080F022AA82BA03004005EA249C5001220A
:100E0C00740F5AFBBB03028007740F5AFBBB0B45D4
:100E1C00A2AF9203C2AFEA2400F582E43400F5835A
:100E2C007402F07B0074012AFCE43BFDEC2400F519
:100E3C0082ED3400F583E51CFCF074022AFAE43BE5
:100E4C00FBEA2400F582EB3400F583AA1B7B00EA55
:100E5C00F0A20392AF22E582FA2483500122EA54D5
:100E6C0003600122A2AF9204C2AFEA2400F582E42F
:100E7C003401F5837402F07B0074012AFCE43BFD21
:100E8C00EC2400F582ED3401F583E51CF074022AA4
:100E9C00FAE43BFBEA2400F582EB3401F583AA1B50
:100EAC00EAF0A20492AF22AA82BA80004005EA249A
:100EBC004B500122EA5403600122A2AF9205C2AF4B
:100ECC00EA2480F582E43400F5837402F07B00742C
:100EDC00012AFCE43BFDEC2480F582ED3400F58323
:100EEC00E51CF074022AFAE43BFBEA2480F582EB61
:100EFC003400F583AA1BEAF0A20592AF22C2E8C225
:100F0C00EA751B00751C01758243120DFF751B8061
:100F1C00751C00758253120DFF0090E650E4F00032
:100F2C0090E652E4F00090E654E4F00090E656E4CB
:100F3C00F00090E65174FFF00090E65374FFF0005F
:100F4C0090E65574FFF00090E65774FFF00090E6C1
:100F5C0058E4F090E65974FFF090E65AE4F090E60D
:100F6C005B74FFF090E65CE4F090E65D74FFF0904B
:100F7C00E65EE4F090E65F74FFF00090E660E4F06B
:100F8C000090E66174FFF090E662E4F090E6637422
:100F9C00FFF090E665E4F090E668740BF05391AFC7
:100FAC00D2E8D2EA2222AA82120FB1DAFB2290FBFB
:100FBC0050A3E582458370F922AA82AB83120FBA43
:0A0FCC001ABAFF011BEA4B70F42271
:0D0FE400758121120954E5826003020FDFC0
:00000001FF
